:10000000000004308A00572CA50084178004841354
:10001000FA30B200B3010522A60AAF0AAA01AB0169
:1000200000082505B200000000082505B3003206CF
:10003000330525060319AA0A0319AB0A3308B200CF
:10004000AE030319AF030319A60B13282A081B2AB2
:100050008030A100FE306421013064217530A7009A
:100060003030A429A101A117B600B608031D3A2813
:1000700003013B280130B6020310A20CA20CA20C13
:10008000C0302205403EB607FE30642136086429A0
:10009000A101A117B600FE30642136086429A01121
:1000A00024080319A0150530A3002730AB00103039
:1000B00065200330AB00E8306520AB01643065207B
:1000C000AB010A3065202E086C28AA002F08A70073
:1000D0002E08A600E9212608A600A3030319A011F3
:1000E000240803197628230203187D282608031DF7
:1000F000A011A0197D28303E64290800CA00BA1F4B
:1001000083282D306421BC0F8A28BB0F8A28BA0AA5
:100110000319BA0AC101C201C301C401BA176A3086
:10012000B9070310BA0CBB0CBC0CC40CC30CC20C3A
:10013000C10CB90F91283C083902BC07B9023B0831
:100140003A02BB07BA02A401DE202E306421CB01A3
:100150000310410DBC00420DBB00430DBA00440D1D
:10016000B900CB0D0310BC0DBB0DBA0DB90DCB0DF5
:100170004108BC0742080318420FBB074308031895
:10018000430FBA0744080318440FB9070318CB0FED
:100190000310BC0DBB0DBA0DB90DCB0D4B08303E95
:1001A00064213C08C1003B08C2003A08C30039087A
:1001B000C400CA0BA72803101B2A0621A01124087B
:1001C000031DE528A0150A30A4003C08A9003B083F
:1001D000A8003A08A7003908A600A301B101B001A0
:1001E000AF010A30AE00B321A30A23082402031D85
:1001F000EE282E08031DA011A01D0029240B0329A1
:100200002E08303E6421A40BE5281B2ABC1F0800E1
:10021000B909BA09BB09BC09B90A0319BA0A031911
:10022000BB0A0319BC0A2D306429B30006118611DC
:100230008316061186110F30860583123308A01825
:100240003F293E30A7008030A4213330B200532133
:100250001330A7008830A42153216430A3215321F7
:100260006430A3212230B200532128303E210C30CB
:100270003E2106303E21A01433083F292014B2004D
:10028000201C4D298611033C031C522952210730A2
:10029000A700D030A421031408002014FE3C031949
:1002A00062298615201C201006150F30860532089D
:1002B000F039860400000611B20E00002018532900
:1002C0003230A32133081B2AA11B15290800A300E3
:1002D000CC01230803178D000313240803178F0094
:1002E0007A2103191B2A6421A30A0319A40ACC0F3B
:1002F00069291B2A831603178C170C1400000000B1
:1003000083120C081B2AB200B20DB20D320D38391F
:10031000C1389F003230A3211F151F198D291E08D7
:10032000BA0083161E088312B9001B2AAB01AA006B
:10033000FF30AA07031CAB07031C1B2A0330A700CE
:10034000E630A4219829A701FC3EA600A709031CBA
:10035000AF29FF300000A6070318AA29A60700004E
:10036000A70FA9290800BD01BE01BF01C0012130AE
:10037000AC00DA29BD0DBE0DBF0DC00D2E083D022B
:100380002F08031C2F0F3E023008031C300F3F02C2
:100390003108031C310F4002031CDA29C0002E086B
:1003A000BD022F08031C2F0FBE023008031C300FA4
:1003B000BF020314A60DA70DA80DA90DAC0BBA29F9
:1003C0004008B1003F08B0003E08AF003D08AE0055
:1003D0001B2AAF01AE011030B200270DAE0DAF0DDC
:1003E0002A08AE022B08031C2B0FAF020318FF29AB
:1003F0002A08AE072B0803182B0FAF070310A60D12
:10040000A70DB20BED29260808001030B800A7018F
:10041000A601B30CB20C031C132A2A08A6072B084A
:1004200003182B0FA707A70CA60CAF0CAE0CB80B2C
:10043000092A2E08080083138312031308004208B8
:100440004606D000D01B582AC21B3F2A410845024D
:10045000031C0034031D013442084602031C00340F
:10046000031D013443084702031C0034031D0134FB
:1004700044084802031C0034031D013400344508BD
:100480004102031C0034031D013446084202031CD0
:100490000034031D013447084302031C0034031DCC
:1004A000013448084402031C0034031D01340034A5
:1004B000C61F0134003446084206D000D01B902AE3
:1004C000C61B792A45084102031C0034031D013470
:1004D00046084202031C0034031D0134470843024E
:1004E000031C0034031D013448084402031C00347B
:1004F000013441084502031C0034031D0134420845
:100500004602031C0034031D013443084702031C48
:100510000034031D013444084802031C0034013434
:10052000C21F013400348030C60645084102CA00AB
:100530000318B42ACA09CA0A4108CF004508C100F5
:100540004F08C5004208CF004608C2004F08C60049
:100550004308CF004708C3004F08C7004408CF0036
:100560004808C4004F08C8001A304A0203181B2A62
:10057000C50803191B2ABD014208CF004606CE005C
:10058000C217C6170830CA02031CCE2A4808BD008D
:100590004708C8004608C700C601C22ACA0703198F
:1005A000DA2A0310C60CC70CC80CBD0CCA03CA0853
:1005B000031DD12ACE1F212B4808C4024708031C63
:1005C000470FC3024608031C460FC2020318F22A53
:1005D000C209C309C409C40FF02AC30A0319C20A15
:1005E0008030CF06BD09BD0A0319FD2AC403440F9C
:1005F000FD2AC303430A0319C2030430CA00C20818
:10060000031D112B4308C2004408C3003D08C40069
:10061000BD010830C102031C402BCA030319402B43
:10062000FF2AC21B1C2B0310BD0DC40DC30DC20D30
:10063000C1030319402B112BBD1F202BBD01362BED
:100640003F2B4808C40747080318470FC30746084D
:100650000318460FC207031C342BC20CC30CC40C76
:10066000BD0CC10A0319422BBD1F3F2BC40F3F2BEA
:10067000C30F3F2BC20F3F2B031441102D2B492BCF
:10068000C101452BCD16FF30C100C401C30180302C
:10069000C200CF1B4C2BC2131B2A4208BF004606C8
:1006A000CE004108003A031D4508003A03199D2B6E
:1006B000C1077E30031C602BC10203189F2B632BE4
:1006C000C102031C9C2B4408BD004308BE00BF1799
:1006D000C617C401C301C2011830CF00BF0CBE0C45
:1006E000BD0C031C7D2B4808C40747080318470F9F
:1006F000C30746080318460FC207C20CC30CC40C3C
:10070000CF0B6E2BC21B8C2BC40DC30DC20DC108A9
:1007100003199C2BC1033F0D031C9B2BC40F9B2B68
:10072000C30F9B2BC20F9B2B0314C20CC30CC40C16
:10073000C10A03199F2BA62B4D15C101A22BCD1465
:10074000FF30C100C401C3018030C200CE1BA92B01
:10075000C2131B2A4108CF004208C1004408C2004E
:100760004108C400C40DCF0CC40CCD01C40DCF0D85
:10077000031CC52B4D158030CD06031DC52B4D1414
:10078000CF01C401C301C201D22B4F0A0319CB2BE5
:100790000314C40CD22B0310C40C031DD12BCD1495
:1007A000CD1CCD15CD19D82BCD1CE52B4D19DF2B2C
:1007B0007F30C400FF30C300C200C1000A2C80306B
:1007C000C400E32BC4010030DB2B4D18E22BC10128
:1007D0009F304F020318D62B7E304F02031CE22BB2
:1007E0009E304F020319FB2B0310C40CC30CC20C28
:1007F000C10CCF0AF02B4D1D0A2CC109C209C30937
:10080000C409C10A0319C20A0319C30A0319C40A95
:10081000C41FE22B41081B2AC301C401CE131F2CA5
:10082000CE13C41F1F2CC409C309C209C109C10FBB
:100830001E2CC20F1E2CC30A0319C40ACE179630F1
:10084000CF00C40803192D2C0830CF074208C1007F
:100850004308C2004408C300422CC308031D422CB5
:100860000830CF024208031D3E2C0830CF02410859
:10087000031D3D2C4408CF004C2CC101C30041088E
:10088000C200C101C31B4A2C0310C10DC20DC30D10
:10089000CF03422CCE1FC3134108C4004F08C10030
:1008A0004308CF004208C3004F08C2001B2A83122E
:1008B00003134030CD00A00183169B0107309C003C
:1008C000063085000330860004309B0080309F0096
:1008D00007309C00FE3083128A01152140308A01C6
:1008E00015210E308A01152111308A011521103091
:1008F0008A01152110308A01152110308A01152135
:1009000015308A0115210E308A01152100308A0127
:100910001521FE308A01152148308A0115210A303F
:100920008A0115210E308A01152111308A01152105
:1009300011308A01152111308A01152111308A01E7
:1009400015210E308A01152100308A011521FE3053
:100950008A01152150308A0115210A308A0115219A
:1009600011308A01152111308A01152111308A01B7
:10097000152111308A01152111308A0115210E30FF
:100980008A01152100308A011521FE308A011521C6
:1009900058308A01152104308A0115210E308A0150
:1009A000152104308A01152104308A0115210430F3
:1009B0008A01152104308A0115210E308A01152182
:1009C00000308A011521FE308A01152160308A012C
:1009D00015210E308A01152111308A0115211030A0
:1009E0008A0115210E308A01152101308A01152155
:1009F00015308A0115210E308A01152100308A0137
:100A00001521FE308A01152168308A0115210E302A
:100A10008A01152100308A0115210F308A01152124
:100A200010308A01152117308A01152111308A01F1
:100A300015210F308A01152100308A011521FE3061
:100A40008A01152178308A01152100308A0115218B
:100A500000308A01152109308A01152109308A01E7
:100A6000152109308A0115210E308A01152108301F
:100A70008A011521FE308A01152170308A01152165
:100A80000C308A01152112308A01152112308A0199
:100A900015210C308A01152100308A011521003002
:100AA0008A01152100308A01152100308A011521A3
:100AB00064308A0196218A012820D601D501DA0105
:100AC000D901D801D701DE01DD01DC01DB01E20142
:100AD000E101E001DF01E401E301E701E4018A153E
:100AE00034228030A1008A0148200B30A4006230FB
:100AF0008A01672101308A0115214C308A011521B4
:100B000000308A01152102308A0115214D308A01F9
:100B1000152102308A0115210730AB00D0308A013F
:100B200097218A0128208030A100C0308A01482006
:100B300043308A01152150308A01152153308A0132
:100B40001521C6308A01482043308A0115215030D2
:100B50008A0115214D308A011521CA308A014820A9
:100B600007308A01152153308A01152176308A0118
:100B700015212F308A01152168308A0115218A112B
:100B80008618492E0330AB00E830AA0005308400F7
:100B900002308A010420D5002B08D600033056020B
:100BA0008A11031CDB2D8A11031D422FE8305502E8
:100BB0008A110318422F803083120313A100CF3013
:100BC0008A0148202A308A011521D6088A11031D7E
:100BD000002E0A3055028A110318002E8030A10021
:100BE0008A01482020308A0115218A011521A4019B
:100BF0005508AE005608AF008A014F208A11242EF6
:100C0000D6088A11031D192E643055028A11031863
:100C1000192E8030A1008A01482020308A01152138
:100C2000A4015508AE005608AF008A014F208A1172
:100C3000242E8030A1008A014820A4015508AE006E
:100C40005608AF008A014F20E40A5508D707560816
:100C50000318560FD807003003180130D9070030A9
:100C600003180130DA073C3064028A11031D3A2E62
:100C70008A114D2632308A0196218030A100CF3072
:100C80008A01482020308A0115218A01932D8A018A
:100C9000BF2D8A0128208A11DA2FDA088A11031D54
:100CA000792ED9088A11031D792ED8088A11031DBF
:100CB000792E5708083C8A11031C792E8030A10038
:100CC00084308A01482020308A0115218A011521AB
:100CD0008A0115218A011521A4015A08BC0059086E
:100CE000BB005808BA005708B9008A01DE208A11F3
:100CF000072FDA088A11031DA32ED9088A11031DB4
:100D0000A32ED8088A11031DA32E5708623C8A110E
:100D1000031CA32E8030A10084308A01482020309B
:100D20008A0115218A0115218A011521A4015A0879
:100D3000BC005908BB005808BA005708B9008A011E
:100D4000DE208A11072F59085A048A11031DCE2E5E
:100D5000033058028A11031CB52E8A11031DCE2EB2
:100D6000E73057028A110318CE2E80308312031306
:100D7000A10084308A01482020308A0115218A018F
:100D80001521A4015A08BC005908BB005808BA0034
:100D90005708B9008A01DE208A11072F59085A0422
:100DA0008A11031DF72E273058028A11031CE02EEA
:100DB0008A11031DF72E0F3057028A110318F72EE0
:100DC000803083120313A10084308A014820203030
:100DD0008A011521A4015A08BC005908BB00580813
:100DE000BA005708B9008A01DE208A11072F803027
:100DF000A10084308A014820A4015A08BC00590887
:100E0000BB005808BA005708B9008A01DE205A080A
:100E1000C4005908C3005808C2005708C1008A011D
:100E200010241130C800C730C7003A30C6007730F0
:100E3000C5008A014D234408DE004308DD00420856
:100E4000DC004108DB008030A1008A308A014820A4
:100E50005E08BC005D08BB005C08BA005B08B90016
:100E600002308A017E20E401DA01D901D801D701DC
:100E7000DE01DD01DC01DB01D601D50132308A0162
:100E8000962108008A0128208030A10085308A013F
:100E9000482059308A01152102308A0115210B3072
:100EA000A4006D308A0167218030A100C1308A0121
:100EB00048200B30A40077308A0167210330AB0053
:100EC000E9308A0197218A012820013086180030F4
:100ED000C900033056028A11031C762F8A11031DA4
:100EE000782FE83055028A110318782F0301031D6B
:100EF000013083120313C9058A110319D62F033059
:100F0000AB00E830AA000530840002308A010420DA
:100F1000D5002B08D6008030A1008A01482043303C
:100F20008A01152150308A01152153308A0115217B
:100F30003A308A011521A4015508AE005608AF00C9
:100F40008A014F208030A100C0308A01482007303C
:100F50008A01152153308A01152176308A01152125
:100F60002F308A01152168308A0115213A308A0113
:100F700015215508C1005608C2008A010C24A03072
:100F8000C8001A30C7002F30C6007D30C5008A0166
:100F90004D234408BC004308BB004208BA00410886
:100FA000B90002308A017E208A01652F8A0128203B
:100FB0008A01932D8A0128208030A1008A014820CF
:100FC00055308A01152156308A01152120308A01B9
:100FD000152101308A0115214C308A01152100307C
:100FE0008A01152102308A0115214D308A0115210F
:100FF00002308A0115210130AB00F4308A019721BB
:101000008A0128208A150618302A02308A01832195
:101010003A08C2003908C1008A010C244408D400EF
:101020004308D3004208D2004108D100C401C301E3
:10103000C2017F30C1005408C8005308C7005208DD
:10104000C6005108C5008A0195224408D40043080F
:10105000D3004208D2004108D100C401C3012030AE
:10106000C2008130C1005408C8005308C7005208AC
:10107000C6005108C5008A014D234408BC0043083E
:10108000BB004208BA004108B9003C08D4003B0844
:10109000D3003A08D2000A3039028A1503185228C0
:1010A0004D150030D1001E308A019621A430C800B1
:1010B0007030C7007D30C6007E30C5005408C400C3
:1010C0005308C3005208C2005108C1008A0193228C
:1010D0004408BC004308BB004208BA004108B900FC
:1010E000CD30C400CC30C3000430C2008230C10017
:1010F0003C08C8003B08C7003A08C6003908C500CC
:101100008A014D234408D4004308D3004208D2008A
:101110004108D100C401C3012030C2008230C100A7
:101120005408C8005308C7005208C6005108C5003B
:101130008A015B22013C8A150319A0280D30E800C2
:101140005408C4005308C3005208C2005108C1002B
:10115000C801C7012030C6008230C5008A015B2269
:10116000013C8A150319BE280E30E8008030A1002A
:101170008C308A01482020308A0115218030A1005E
:101180008A01482055308A01152156308A011521DF
:1011900020308A01152103308A0115214E308A0141
:1011A000152144308A01152145308A0115214B3023
:1011B0008A01152153308A01152103308A01152136
:1011C00020308A0115213A308A0115210130A20010
:1011D00068088A0134205408BC005308BB00520838
:1011E000BA005108B9005408C4005308C30052089B
:1011F000C2005108C1008A01AA23B9004208BA00FE
:101200004308BB004408BC00A4018A01DD20540847
:10121000C4005308C3005208C2005108C100C801ED
:10122000C7014030C6008030C5008A015B22013C06
:101230008A15031943298030A100C0308A01482053
:1012400044308A01152102308A01152104308A01B7
:10125000152102308A0115214B308A0115212030D9
:101260008A01152153308A01152145308A01152143
:1012700056308A01152103308A0115210B30A40054
:1012800087308A0167215408C4005308C3005208FC
:10129000C2005108C100C801C7014030C6008030FB
:1012A000C5008A015B22C9005408C4005308C3006A
:1012B0005208C2005108C100C801C7014030C60031
:1012C0008130C5008A011F22C9058A1503197A29B0
:1012D0008030A100C0308A0148200B30A4008E303D
:1012E0008A01672103308A0115210B30A400973051
:1012F0008A0167215408C4005308C3005208C20081
:101300005108C100C801C7014030C6008130C50086
:101310008A015B22C9005408C4005308C300520864
:10132000C2005108C100C801C701C6018230C50012
:101330008A011F22C9058A150319B6298030A10028
:10134000C0308A01482059308A01152102308A01B3
:1013500015210B30A4009F308A01672103308A01D8
:1013600015210B30A40087308A0167215408C4007E
:101370005308C3005208C2005108C100C801C70188
:10138000C6018230C5008A015B22C9005408C4002E
:101390005308C3005208C2005108C100C801C70168
:1013A0003030C6008230C5008A011F22C9058A1567
:1013B0000319F6298030A100C0308A01482000308E
:1013C0008A0115214F308A0115214B308A011521E0
:1013D00020308A01152159308A01152102308A01F5
:1013E00015210B30A400A8308A016721C401C30174
:1013F0003030C2008230C1005408C8005308C70012
:101400005208C6005108C5008A015B22013C8A15BA
:1014100003192B2A8030A100C0308A0148204130B6
:101420008A01152104308A0115210B30A400B33044
:101430008A01672103308A0115214B308A01152169
:101440008A01152141308A01152154308A01152164
:1014500021308A011521C8308A0196218A15022877
:101460008A0128208A01712D1030E30002306302C6
:101470008A15031C572A8030A1000130A20063089E
:101480008A0134202A308A0115218030A1000130E0
:10149000A200630A8A01342020308A0115212D30F0
:1014A0008A0196210130E3028A150318362A10308A
:1014B000E300043063028A15031C7A2A8030A100FD
:1014C0000130A20063088A01342054308A011521BA
:1014D0008030A1000130A200630A8A01342020304C
:1014E0008A0115212D308A0196210130E3028A15E7
:1014F0000318592A1030E300063063028A15031CD2
:101500009D2A8030A1000130A20063088A013420A6
:1015100041308A0115218030A1000130A200630A08
:101520008A01342020308A0115212D308A0196212C
:101530000130E3028A1503187C2A1030E3000830DA
:1015400063028A15031CC02A8030A1000130A2006A
:1015500063088A01342032308A0115218030A100CD
:101560000130A200630A8A01342020308A0115214B
:101570002D308A0196210130E3028A1503189F2A33
:101580001030E3000A3063028A15031CE32A80301E
:10159000A1000130A20063088A01342045308A018D
:1015A00015218030A1000130A200630A8A01342095
:1015B00020308A0115212D308A0196210130E30265
:1015C0008A150318C22A1030E3000C3063028A1512
:1015D000031C062B8030A1000130A20063088A01A1
:1015E000342049308A0115218030A1000130A20049
:1015F000630A8A01342020308A0115212D308A01A6
:1016000096210130E3028A150318E52A1030E30021
:101610000E3063028A15031C292B8030A100013093
:10162000A20063088A0134202A308A011521803003
:10163000A1000130A200630A8A01342020308A010F
:1016400015212D308A0196210130E3028A150318F5
:10165000082B8030A1008E308A01482020308A017A
:1016600015218A0115210330AB0020308A01972112
:101670008030A1008A0148200B30A400BC308A01D0
:1016800067218030A100C5308A01482001308A01DD
:1016900015214C308A01152100308A0115210230B4
:1016A0008A01152143308A01152102308A01152152
:1016B0000730AB00D0308A0197218A01282008002A
:1016C0008A15602B5200410044005900410053002C
:1016D00059004F004E00200000004B005300450011
:1016E0004B002000200020002000200000005200BD
:1016F0004100440059004100530059004F004E0082
:1017000020002100210021002000200000005900BD
:101710004500200055005600200000004F005200F8
:1017200054004100200053004500560000005900BD
:1017300045002000550056002000200000004B000E
:10174000530045004B0020005300450056000000A8
:101750004B00530045004B00200055005600200070
:1017600020002000000049005200490020005500E0
:10177000560020004400000052004100440059007F
:101780004100530059004F004E0020005600450014
:08179000200055005600000086
:02400E00223F4F
:00000001FF
